:020000020000FC
:100000000C9456000C94AA0D0C94AA0D0C94AA0DF5
:100010000C94AA0D0C94AA0D0C94AA0D0C94AA0D84
:100020000C94AA0D0C94AA0D0C94AA0D0C94AA0D74
:100030000C94AA0D0C94AA0D0C94AA0D0C94AA0D64
:100040000C94AA0D0C94AA0D0C94AA0D0C94AA0D54
:100050000C94AA0D0C94AA0D0C94AA0D0C94AA0D44
:100060000C94AA0D0C94AA0D0C94AA0D0C94AA0D34
:100070000C94AA0D0C94AA0D0C94AA0D0C94AA0D24
:100080000C94AA0D0C94AA0D0C94AA0D0C94AA0D14
:100090000C94AA0D0C94AA0D0C94270C0C94AA0D88
:1000A0000C94AA0D0C94AA0D0C94AA0DA8950FEF10
:1000B0000DBF0AE00EBF0E94FA0C0E9482027894E3
:1000C0000E943A010FEFC02E0E94FF000E949E0185
:1000D0000C945F000590002009F0089500E0009363
:1000E000BD050C94E207E6E5FBE10E946A000716F5
:1000F00071F40E946A00061659F40E946A000516FF
:1001000041F431960591F491E02F099508953196C7
:10011000319630960C94750070EF60EF41E01881D5
:100120000E94C300013021F40E94B7000C948C009F
:10013000512F0E94B7001D30A9F03D2C18811D30B1
:1001400089F00E94C3003D1441F4762F652F512F92
:100150000E94B7004395433089F718810E94C3007D
:100160003D1409F008950E94B7000C94AD00DB1512
:1001700041F4CA1531F404E00093BD050C94E20784
:100180000895219708951F9300271D3011F40C94B2
:10019000E6001F75103011F40C94D0001C3019F4D7
:1001A00001E00C94E700103112F40C94E7001B35C9
:1001B00012F00C94E70010341AF003E00C94E700FE
:1001C0001A3112F422F402E00C94E70004E0D02E7D
:1001D0001F910895CF3329F447E00E9428010C9421
:1001E000040148E00E94410140E20E944101412F88
:1001F0000E944101C3951DE018830C9404014EE355
:100200000E942801D5E0CFE30E944801183011F385
:100210001F3701F31A3011F40C94040118831D30B8
:1002200069F0C03029F447E00E9428010C940401D1
:10023000CA95412F0E9441010C94040108950E9427
:100240004A028F93492F0E9428014F9101D00895AF
:100250000090C80005FE0C9428010E940906B6FF14
:100260000C9437010090C80007FEFCCFBF7B409381
:10027000CE0008954DE00E9428014AE00E94280126
:1002800008954D3019F40E943A0108950C94280104
:10029000889500000091C80007FF0C944801109158
:1002A000CE0008950E9457010E943A010895459199
:1002B000442321F1483F21F40E947F010C9457010F
:1002C000493F31F4159045910E9499010C945701D2
:1002D0004A3F21F40E943A010C9457014B3F51F4DC
:1002E000EF93FF93E4ECF0E20E945701FF91EF914E
:1002F0000C9457010E9428010C9457010895EF9324
:10030000FF93112445914A3049F04C3039F04A3F6F
:1003100029F0493F19F013940C9482011A944CE38C
:10032000141A1194169440E20E949901FF91EF91E2
:1003300008950E9428011A94E1F70895D5E0CFE3CB
:100340000FEFA02E05E0B02E18810E94C3000230EE
:1003500011F40C9486060E943A01A1600C94B1013C
:10036000AE7F8DB78F3C28F408E00093BD050C9458
:10037000E2070E948C005D30F9F05B33E9F0032D59
:10038000023049F47F706F705F700E9465020E94B6
:10039000F2010C94B1017F756F755F75413039F4CE
:1003A000032D033021F40E94DE010C94B1010E9460
:1003B00073005D3009F00895A160089551545A31D9
:1003C0002AF005E00093BD050C94E207505CA0FF05
:1003D00019F40E94F2010895F5E0E52F50810E9482
:1003E000F20108950F93F4E0EC2D5083CA940C2D84
:1003F000033F28F406E00093BD050C94E2070F913B
:1004000008950F93C3940C2D00302AF007E0009359
:10041000BD050C94E207F4E0EC2D50810F91089596
:100420000E94010207E005175AF001E0503021F068
:10043000000F5A950C941602502F0E94F201089555
:100440000AE00093BD050E94E207703049F0705D3C
:10045000472F0E942801603019F440E30E942801D0
:10046000603021F0605D462F0E942801505D452FCD
:100470000E942801089577276627545618F073952F
:100480000C943D025C595A5018F063950C94430249
:10049000565F0895982F9695969596959695905DAA
:1004A0009A3308F0995F8F70805D8A3308F0895F16
:1004B000089596FD975F9F7086FD875F8F70990FF7
:1004C000990F990F990F892B08957330B2F47230F8
:1004D00032F0663092F4653012F0563072F46623D2
:1004E00021F00AE0500F6A9581F7772309F4089507
:1004F00004E68894500F7A95C0F701E00093BD059B
:100500000C94E207E0E6FEE10E94520108950E9489
:100510003A01F4E0E4EFC091B905D091BA05FD17B6
:1005200011F4EC1731F040810E94410131970C9495
:100530008F020E943A010E943A01E0E9F0E20E9433
:1005400057015091B9057091BA05505071400E9401
:10055000F201572F0E943B020E942502EEE9F0E2D1
:100560000E9457010E9401020E943B020E94250244
:100570000E943A010895AE7F0E94B1010E940102DB
:100580000E943B020E9425020E943A0108950E94A7
:10059000B00144E20E9428010E940102852F0E94BE
:1005A0001F010E943A010895AE7F0E94B1010E948E
:1005B0000102052F0E940102F5E0E52F0083089556
:1005C000A2FF0C949203AE7F0E94B1010E9401022F
:1005D000452E0E940102652F0E940102552EF5E072
:1005E000E52F6083A062A860AA7F0895F5E0E52D5D
:1005F0000081041519F003950083A06108950E94FD
:10060000B0010E940102052F0E940102501721F043
:1006100055270E94F20108955FEF0E94F2010895AC
:100620000E94B00150E000B605FE51E00E94F201C8
:1006300008950E94B0010EEF0C1949F00E940102CA
:100640005F930E940102F52FEF910C942B030E94FF
:100650000102E52FFF2750810E94F20108950E94B8
:10066000B0010DEF0C1961F00E9401025F930E942E
:1006700001025F930E940102FF91EF910C944703E6
:100680000E940102052F0E940102E02FFF275083E4
:1006900008950E94B0010E940102052F0E940102EC
:1006A000509F1120F09921F4502D0E94F2010895DD
:1006B0000FE00093BD050E94E2070E94B0010E9476
:1006C00001025523F099B9F0052F0E940102652F10
:1006D000771B59E0661F5A9551F0771F701B20F465
:1006E000700F88940C946A0308940C946A03562F34
:1006F0000E94F201089501E10093BD050E94E20706
:100700000E94B0010E940102052F0E940102500FB9
:10071000F09918F00E94F20108950FE00093BD05D2
:100720000E94E2070E94B0010E940102052F0E9470
:100730000102501BF0991BF00E94F201089500E1A4
:100740000093BD050E94E2070E94B0010E940102D1
:10075000052F0E94010250230E94F20108950E9479
:10076000B0010E94010256950E94F20108950E9474
:10077000B0010E940102550F0E94F20108950E94EB
:10078000B0010E940102052F0E940102502B0E941D
:10079000F20108950E94B0010E940102052F0E94FB
:1007A000010250270E94F20108950E94B0010E94A8
:1007B000010250950E94F20108950E94B0010E942A
:1007C000010251950E94F201089551E00E94F20148
:1007D00008950E94B0010E940102052F0E940102AB
:1007E00050170C94FB030E94B0010E940102052FD8
:1007F0000E940102051750E042F739F30E94F2010E
:1008000008950E94B0010E940102552309F0A260E0
:1008100008950DB70E5F0DBF0895A46008950E945E
:10082000B0010895B260089598810E94B700888150
:100830000E945902582F0E94F2010E94B7000E94A4
:10084000B00108950E94B0010E940102CF93DF938E
:10085000D8ECC9EFCA950000E9F7DA950000C9F7AE
:100860005A95B1F7DF91CF91089555270E94F20173
:100870000E94B0010E94010201E005172AF0F098E1
:1008800050FF0895F09A08950CE00093BD050E9472
:10089000E2070E94B0010E940102452FF4E0E4EF5C
:1008A0008091B9059091BA050C946104F91711F47F
:1008B0008E1708F500810D3019F031970C9456040D
:1008C0003197552766277727F91711F48E1798F473
:1008D00010810E94C300023031F4762F652F512F12
:1008E00031970C9464047F706F705F700E94650292
:1008F0004517E1F6089509E00093BD050C94E20761
:100900000E944904DF2FCE2F08950E944904A06C55
:100910000895B2FF0C948E04B1600895B2600895FA
:100920000E94B0010E940102452F0E9428010895F3
:10093000889500000091C80007FFFACF5091CE00C3
:10094000533009F4B2600E94F20108950E94B00190
:100950000E94010208E040E3551F08F441E378DCFF
:100960000A95C9F70E943A01089504EB5091BE051B
:10097000579508F450275093BE050E94F201089540
:10098000D4E0C4EF0FEFC02EA1600E940906A5FFBE
:100990000C94CD046C2E7D2EAF7DA4FF0C94D3045B
:1009A000D72DC62DAF7EA6FF0C94DB04D093BC05DB
:1009B000C093BB05AF7BA7FF0C94E204DF2FCE2FC3
:1009C000B460AF77B0FF0C94EA04C091BB05D0913E
:1009D000BC05BA7FB1FF0C94F4040E940406C091D8
:1009E000B905D091BA05BD7F0091BA05D01721F4A1
:1009F0000091B9050C17A0F418810E94C300A1FF53
:100A00000C940705043019F021970C94C204AD7FB3
:100A1000023019F421970C94C2040E94B101B2CFA4
:100A20000895F4E0E4EFF093BA05E093B9050FEF11
:100A3000C02EAA27BB27F1E0E0E000E00193F430EC
:100A4000E8F3E43FD9F7F5E0E0E400E00193F530A6
:100A5000E8F3EA35D9F70E943A01E8E1FEE10E94A5
:100A600052010895E0EDFFE10E945701EAEFFFE136
:100A70000E94570100E1202EF4E0E4EF8F2F0E9446
:100A80001F018E2F0E941F014AE30E94280140E2AD
:100A90000E942801F13011F4E030D9F080810E94E9
:100AA0001F0140E20E94280131972A9481F40E949C
:100AB0003A018F2F0E941F018E2F0E941F014AE3CF
:100AC0000E94280140E20E94280100E1202E0C949F
:100AD0004A050E943A010E943A01E6E1F0E20E94D2
:100AE00057018091BA050E941F018091B9050E94AB
:100AF0001F010E943A01E0EDFFE10E9457010E94B0
:100B00003A010895E0EDFFE10E945701EAEEFFE1AE
:100B10000E94570100E1202EF3E0EFEF8F2F0E949B
:100B20001F018E2F0E941F014AE30E94280140E20C
:100B30000E9428010F93E03000E0F0070F91F1F0E0
:100B4000F2BDE1BDF89A80B50E941F0140E20E940B
:100B5000280131972A9481F40E943A018F2F0E9434
:100B60001F018E2F0E941F014AE30E94280140E2CC
:100B70000E94280100E1202E0C949A050E943A015F
:100B8000E0EDFFE10E9457010E943A010895E0ED77
:100B9000FFE10E945701E6EDFFE10E94570100E1ED
:100BA000202EE0E4F5E08F2F0E941F018E2F0E947F
:100BB0001F014AE30E94280140E20E942801EA3511
:100BC000D1F081910E941F0140E20E9428012A94E5
:100BD00081F40E943A018F2F0E941F018E2F0E94E4
:100BE0001F014AE30E94280140E20E94280100E11F
:100BF000202E0C94DF050E943A01E0EDFFE10E94F7
:100C000057010E943A010895E8E8F0E20E94570176
:100C100008950090C80007FE0C9419060091CE00BC
:100C2000033111F4B06408950091CE00033009F44B
:100C3000B2600895DF93D5E0DA950000E9F7DF911F
:100C40000895DF93D2E3DA950000E9F7DF91089584
:100C5000CF93DF93D8ECC3EFCA95000000000000EB
:100C60000000D1F7CFEFCA95000000000000D9F7CF
:100C7000CCEFCA950000000000000000D1F716F08C
:100C80006894E9CFDA95E89431F7DF91CF91089530
:100C9000D5E0CFE3552788279927BF7D1881CA95CE
:100CA00083951D3051F00E94C300023041F0B062C4
:100CB0000130A1F393950C944E06092F0895B5FFCA
:100CC00053950C944E0604E00093BD050C94E20786
:100CD00002E00093BD050C94E2070BE00093BD0514
:100CE00071C17F706F705F700E9465020895D5E0DA
:100CF000CFE3E03069F308810083319721970D300D
:100D0000C1F7F093BA05E093B90508950E9448062B
:100D1000543018F78091B9059091BA05943021F4B8
:100D2000843F11F40C94F506D5E0CFE355276627F0
:100D30007727CA1542F218810E94C300023031F4AD
:100D4000762F652F512F21970C9499060E947106DA
:100D5000452EE091B905F091BA05B77FBF7E7727A0
:100D60006627552755243196F43011F4E53F69F094
:100D700010810E94C300043041F0023081F7539487
:100D8000562F672F712F0C94B306052D033031F0C9
:100D90005394562F672F70E00C94C506B4FD0C9445
:100DA000D406B0610C94AF060E9471064516F1F1AD
:100DB00018F4B8607F2E6E2EF43029F4E53F19F454
:100DC000B3FF0C94F506B3FF0C94EA06541538F4FF
:100DD0000C944007F43019F6E53F09F60895F43015
:100DE00021F4E53F11F40C9440070E9448060030BE
:100DF00009F40895D5E0CFE3E091B905F091BA0583
:100E0000F13021F4E03011F40C94110708810083D3
:100E1000319721970D30A1F7F093BA05E093B9050A
:100E2000089502E00093BD050C94E2073197EF01AD
:100E3000D13021F4C03011F40C946306088121975D
:100E40000D30B1F70E2F0C1B8091B9059091BA05AA
:100E5000800F8093B90518F493959093B905D1301C
:100E600011F4C03031F008810083219731970C9440
:100E70002F070E944806003011F00C948606089552
:100E80000E944806003071F10091BA05013029F442
:100E90000091B9050050081720F2E091B905F091D2
:100EA000BA05DF2FCE2FC81BD040D093BA05C09310
:100EB000B905F71521F4E61511F40C9465070081C6
:100EC0000883219631960C945907D5E0CFE3F72D8E
:100ED000E62D3197088100830D3021F0319721975D
:100EE0000C946A070895D4E0CFEFE091B905F09132
:100EF000BA05CE1BDF0BF3E0EFEFEC17FD072CF488
:100F0000E2E3F0E20E9452010895E2E5F0E20E947D
:100F100052010FEFC02E5091B9050E94F20150917D
:100F2000BA050E94F201D4E0CFEFF3E0EFEF0881C1
:100F3000F9990C949807F2BDE1BD00BDFA9AF99AAF
:100F4000D13011F4C03051F031970F93E03000E010
:100F5000F0070F9119F021970C9497070895E4E793
:100F6000F0E20E9452010E941105D4E0CFEFEFEFB2
:100F7000F3E0F9990C94B907F2BDE1BDF89A00B518
:100F80000883D13011F4C03021F0319721970C94AF
:100F9000B9070DEFC02E0E9401025093BA05F52F3C
:100FA0000E9401025093B905E52F0F93EF3F04E033
:100FB000F0070F9131F4E4E6F0E20E9452010E9442
:100FC000110508950E943A010091BD05000FE8EF58
:100FD000FFE0E00F0591F491E02FEE1FFF1F0E944C
:100FE00057010FEF0DBF0AE00EBF0FEFC02EA0E0BC
:100FF000B0E00E943A0163C8661077109310A21007
:10100000C010D610ED100C11361160117A11931129
:10101000AA11C311DC11EF11FC110A1215122312CF
:101020003312441255270E94F2010E94B0010E941F
:10103000010201E00517A2F001E150FD0CE500936B
:10104000B800409A419A00270093B9000095009398
:10105000BB0004E00093BC0004E90093BC000895C9
:101060000CE00093BD050E94E2070091BC0002FF66
:101070000C9464080E94B0010E9401025093BB00CE
:1010800005E80093BC000091BC0007FFFCCF009175
:10109000B900087F083111F0003441F45091B900D3
:1010A0005695569556950E94F2010895003239F0F2
:1010B000083429F002E10093BD050E94E20704E133
:1010C0000093BD050E94E20703E10093BD050E9465
:1010D000E2070091BC0002FF0C9494080E94B0014A
:1010E0000E9401025093BB0005E80093BC000091F0
:1010F000BC0007FFFCCF0091B900087F083241F423
:101100005091B9005695569556950E94F201089552
:10111000003329F002E10093BD050E94E20704E1DB
:101120000093BD050E94E20703E10093BD050E9404
:10113000E2070091BC0002FF0C94C70851E00E9436
:10114000F2010E94B0010E94010201E0051722F1A4
:1011500004EC50FF04E80093BC000091BC0007FFC2
:10116000FCCF0091B900087F003529F45091BB00F5
:101170000E94F2010895003529F002E10093BD05B7
:101180000E94E20704E10093BD050E94E20703E12B
:101190000093BD050E94E2070CE00093BD050E948C
:1011A000E2070091BC0002FF0C94E80804EA0093F7
:1011B000BC000091BC0007FFFCCF0091B900087F84
:1011C000083009F4089502E10093BD050E94E2078A
:1011D00003E10093BD050E94E2070091BC0002FFFD
:1011E0000C94FE0804E90093BC000FEF0093BB00D1
:1011F000089502E10093BD050E94E20703E1009318
:10120000BD050E94E2070091BC0002FF0C941C097E
:101210000091BC0004FF0C94100950E80C941909CB
:101220000091BC0007FFFCCF5091B9005695569530
:1012300056950E94F201089503E10093BD050E94B6
:10124000E20752E00E94F2010E94B0010E940102F6
:1012500003E005174AF0550F550F0E9492090CB58F
:10126000037F052B0CBD08950DE00093BD050E9482
:10127000E2070E94B0010E94010201E0051752F04E
:101280000CB500620CBD50FD0C9449090CB50F7DE6
:101290000CBD08950CE00093BD050E94E2070E947A
:1012A000B0010E94010207E0051782F0052E53707D
:1012B0000CB5087F052B0CBD0DB501600DBD02FC02
:1012C0000C9465090DB50E7F0DBD08950AE00093DD
:1012D000BD050E94E2070E94B0010E940102289809
:1012E000000000005EBD0DB407FE0C9473095EB5EE
:1012F00008952898000000005EBD0DB407FE0C9410
:101300007D095EB50E94F201089551E00E94F2014C
:101310000E94B0010E940102289A50FD0C9491098C
:101320002898089504B1076004B905B1016005B9B2
:1013300001E50CBD0DB50E7F0DBD08950091640053
:101340000E7F0093640000E000937B0055270E940D
:10135000F2010E94B0010E94010200917C00007E17
:1013600060917B006F7D60937B0056FF0C94BB09FE
:1013700060917B00606260937B005F71052B00933E
:101380007C0007EC00937A0000917A0006FD0C9433
:10139000C40907EC00937A0000917A0006FD0C94D2
:1013A000CC09509179000E94F201089555270E94BE
:1013B000F2010E94B0010E94010201E005175AF0FB
:1013C00000917C000F73006250FD0C94E809006CE2
:1013D00000937C0008950CE00093BD050E94E20795
:1013E0000E94740AEF5DFF4F50810E94F201089540
:1013F0000E94740AEF93FF930E94B0010E940102C1
:10140000FF91EF91EF5DFF4F508308950E94740AA2
:10141000EF93FF930E94B0010E9410020E9401020C
:10142000FF91EF91EF5DFF4F0C94790A0E94740ACF
:10143000EF93FF930E94B0010E9410020E940102EC
:10144000FF91EF91EF5DFF4F0C947D0A0E94740AAB
:10145000EF93FF930E94B0010E940102FF91EF9170
:10146000EE5DFF4F508308950E94740AE05EFF4FC7
:1014700050810E94F20108950E94740AEF93FF9335
:101480000E94B0010E9410020E940102FF91EF91A0
:10149000EE5DFF4F0C94790A0E94740AEF93FF935C
:1014A0000E94B0010E9410020E940102FF91EF9180
:1014B000EE5DFF4F0C947D0A0E94740AEF93FF9338
:1014C0000E94B0010E9410020E940102FF91EF9160
:1014D000E05EFF4F0081052350E000230FB601FCC2
:1014E00051E00E94F201089503E05154509FF00131
:1014F00008950081052B00830895509500810523F0
:10150000008308950E94B00101E80093800009E083
:1015100000938100002700938200259A0E94010217
:101520000027009389005093880008950E94B0011D
:1015300003E80093800009E00093810000270093F6
:101540008200259A0E940102052F0E9401025093F9
:101550008900009388000895002700938000089573
:1015600055270E94F2010E94B0010E94010207E08B
:1015700005178AF00091BF05087F502B5093BF05D7
:10158000002700936F0006BB009382000093800049
:101590000093810008950AE00093BD0513DD51E03A
:1015A0000E94F2010E94B0010E94010201E00517B1
:1015B0004AF00091BF050F7750FF01C0006800930B
:1015C000BF0508950CE00093BD05FCDCCF93DF93CD
:1015D0006627552756BB6093850050938400B09AC8
:1015E0000091BF05702F7078C894771F771F7660C1
:1015F0000770EDEFFAE0E00F09947AC006C005C06D
:1016000004C02AC029C028C04FC0033008F005E03C
:10161000709381006093850050938400D4E1C3EF00
:10162000CA950000000000000000D1F7CFEFCA9576
:10163000000000000000D9F7CCEFCA9500000000C0
:1016400000000000D1F716F06894E9CFDA95E8942D
:1016500031F70A9519F74CC00350033008F005E044
:10166000709381006093850050938400D8ECC3EFA1
:10167000CA950000000000000000D1F7CFEFCA9526
:10168000000000000000D9F7CCEFCA950000000070
:1016900000000000D1F716F06894E9CFDA95E894DD
:1016A00031F70A9519F724C0709381006093850083
:1016B000509384000AE0D8ECC3EFCA950000000004
:1016C00000000000D1F7CFEFCA9500000000000035
:1016D000D9F7CCEFCA950000000000000000D1F758
:1016E00016F06894E9CFDA95E89431F70A9519F77E
:1016F0005091840060918500002700938100B0998B
:1017000008C0C9E5D5E068830E94F201DF91CF915E
:101710000895DF91CF910EE00093BD0553DC0E9448
:10172000B0010E940102152F88940E94A70B089512
:101730000E94B0010E940102152F08940E94A70B7D
:1017400008950E94D10B512F0E94F201089504B117
:10175000077E04B905B1086105B979E01C9B0C94BA
:10176000AE0B2D9A259810F02D98259A2C98249A36
:101770000E94F20B24982C9A0E94F20B1C990C9454
:10178000B60B20F02D9A25980C94C80B2D98259A0D
:101790001C9B0C94C80B25982D9A111F7A95F1F675
:1017A000089504B1077E04B905B1086105B979E06F
:1017B0001C990C94D80B88941D9B0C94E70B0894EF
:1017C0002C98249A1D990C94E20B0C94EC0B2C98F9
:1017D000249A1D9B0C94E90B24982C9A111F7A953E
:1017E00039F7089580E590E59A95F1F78A95D9F74C
:1017F0000895CF93DF9355270E94F2010E94B00114
:101800000E9401020517F2F050FD0C94130C0E9487
:10181000DC0CC3ECD5E00993099308835D9A5598D5
:10182000DF91CF910895C7E5D5E00E94530C0027C2
:101830000093C605559A5D980E94B60CDF91CF9132
:10184000789408950CE00093BD050E94E2077F9311
:101850007FB77F936F935F93EF93FF93F4E2E091F1
:10186000C6055091C3056091C4057091C505E50E8C
:10187000F61EE71F5491E093C60550FF0C944A0CE6
:1018800000005D9AFF91EF915F916F917F917FBF13
:101890007F9118955D98FF91EF915F916F917F9186
:1018A0007FBF7F911895C7E5D5E077276627552735
:1018B00000EF102E088001200294002049F080E003
:1018C000581F90E0691F00E0701F0A940C945D0C93
:1018D000099012940120002049F089E9581F99E9E4
:1018E000691F09E1701F0A940C946B0C0880129414
:1018F00001200294002049F08CE5581F9FE8691FE1
:1019000002E0701F0A940C947A0C09901294012042
:10191000002049F089E8581F91E4691F00E0701F1A
:101920000A940C94880C08801294012002940020E0
:1019300049F08DE8581F96E0691F00E0701F0A9477
:101940000C94970C088012940120002041F087EA43
:10195000581F90E0691F00E0701F0A94B1F7509380
:10196000C3056093C4057093C50508950091650093
:101970000F7E00936500002709BB0093BE00009313
:10198000C0000093C1000093CF000093D0000093EB
:10199000C2000093C3000093C40007EC0093D10081
:1019A00000E00093C00001E00093C10000917200CC
:1019B0000064009372000895F894002709BB009317
:1019C000C0000093C1000093BE000093D0000093BC
:1019D000CF000093C2000093C3000093C4000091A5
:1019E00072000F7B0093720000916500006100930C
:1019F00065000895A89504B7007004BF00916000C9
:101A000008610093600000700093600006E204B972
:101A100000E005B900E007B900E008B908E00AB93C
:101A200000E00BB900E00DB900E00EB900E000BB2A
:101A300000E001BB00270093BF050EBBF09A54EBFA
:101A40000091000105270093BE0500E00093CD0042
:101A500000E40093CC0008E90093C90001E003BF53
:101A60005F9A0E9421064F990EC05F980E94AF07AF
:101A70000E94C0040E943A010E943A01E8E1FEE19E
:101A80000E94520108950E9411050895E3E0F0E0DC
:101A900009E007BF049106950370003019F4E0E0F7
:101AA000F8E314C0013019F4E0E0FCE30FC00230A9
:101AB00019F4E0E0FEE30AC0033019F4E0E0FFE3CC
:101AC00005C00BE00093BD050C94E207EF93FF9374
:101AD00008E0102EEE1FFF1F05910F3F19F0003098
:101AE00009F007C01A94C1F705E10093BD050C94F5
:101AF000E207E8EAF0E20E945701FF91EF918F2F91
:101B00000E941F018E2F0E941F010E943A010E9415
:101B10003A011124F8941DBA109268001CBC10BE42
:101B20001FBA10926E0010926F0010927100109206
:101B300072001092C9001092BC0010927A0014B882
:101B400017B81AB81DB810BA15B818B81BB81EB80F
:101B500011BA099418954C495320870252554E20CA
:101B6000C0045052494EBB0250525820C702505236
:101B70004220A604464F52200D044E455854F6020A
:101B800053495A209B024E455720110550500B20B7
:101B9000800350500D20920350500A2049035050AA
:101BA0000F205D03414F56203504454D49549004A4
:101BB000501A1D20D40250501D20E002501C1E203F
:101BC000FF0250501E20F30350501C20E9035049DF
:101BD0004620010450544F200F0450500420140498
:101BE000454E44201204414E4420A4034C5352203D
:101BF000AF034C534C20B703504F5220BF03584FF4
:101C00005220CA03434F4D20D5034E454720DD03E4
:101C1000524E4420B50444454C412204474F544F92
:101C20008004474F53558504524554558904544800
:101C3000454E09044B455920980441434F20100359
:101C40005341564573074C4F4144AF075045454BF0
:101C50001903504F4B452F034F444220F809494484
:101C60004220F00953444220060A43444220160A07
:101C70004F504220260A534242203C0A434242200F
:101C80004C0A494E4220340A494242205C0A4F44E1
:101C90004320F80949444320F00953444320060AED
:101CA00043444320160A4F504320260A5342432000
:101CB0003C0A434243204C0A494E4320340A4942DD
:101CC00043205C0A4F444420F80949444420F00969
:101CD00053444420060A43444420160A4F504420EB
:101CE000260A534244203C0A434244204C0A494EAF
:101CF0004420340A494244205C0A4F444520F809F4
:101D000049444520F00953444520060A43444520F0
:101D1000160A4F504520260A534245203C0A4342AA
:101D200045204C0A494E4520340A494245205C0A68
:101D30004F444620F80949444620F00953444620C0
:101D4000060A43444620160A4F504620260A5342AC
:101D500046203C0A434246204C0A494E4620340A5B
:101D6000494246205C0A44554D5032054544554D84
:101D700082055644554DC70544535245A10B445363
:101D8000434F980B445344458F0B49434720B00AB7
:101D900049434520CF0A49435020E60A50574D3861
:101DA000820A50574520960A50574F20AC0A4444A7
:101DB0005320F90B424C4452460D414443209E09A6
:101DC00041445220D60953504D20210953504F20F1
:101DD0003909535043204F09535057206B09535032
:101DE000522079095350532085095457492012082D
:101DF00054575320D10854575020ED0854574120D0
:101E00003508545757206908545752209908545799
:101E10004220030900000000F93C3DFAF8417474C7
:101E20006F424153494320666F722041546D65678C
:101E30006133325534FAF85665723A20322E313118
:101E4000204275696C6420636F64653A20323031DA
:101E500032303330382E30333133FAF93C2D000034
:101E6000F84F726967696E616C20636F6465202842
:101E700043293230303220627920526963686172BE
:101E8000642043617070656C73FAF8687474703A1A
:101E90002F2F70726F6A656374732E636170706543
:101EA0006C732E6F7267202070726F6A6563747333
:101EB0004063617070656C732E6F726720FAF93C35
:101EC0002DFAF854686520666F6C6C6F77696E67E1
:101ED0002061726520656E68616E63656D656E7404
:101EE000732062792053636F747420566974616C37
:101EF00065FAF86B73765F70726A40676D782E636F
:101F00006F6D20FAF84D65676138382F3136382FFC
:101F10003332382F3332553420706F727420284397
:101F200029323031312C3230313220FAF8545749CD
:101F30002F5350492F444453202620496E70757406
:101F40002043617074757265202843293230313125
:101F500020FAF84D656761333255342055534220DD
:101F6000262044465520426F6F746C6F6164657221
:101F700020737570706F72742028432932303132AB
:101F800020FAF93C2DFAF8416C6C2072696768748C
:101F90007320616E642072656D6564696573206588
:101FA0007870726573736C7920726573657276658B
:101FB00064FAF84E6F7420666F7220636F6D6D6502
:101FC000726369616C20757365FAF93C3DFA000033
:101FD000F9352DFA00005661726961626C657320F3
:101FE000696E2052414D3AFA000045455020436F3A
:101FF0006E74656E74733AFA000050524F47524146
:102000004D204D656D6F727920436F6E74656E74EF
:10201000733AFA0000004E65787420617661696C4D
:1020200061626C65206C6F636174696F6E3A200049
:102030000000FB3A2050726F6772616D20746F6F01
:10204000206C6172676520666F722045455021FAE9
:102050000000536176696E6720746F204545502EED
:10206000FA000000FB4545502065726173656421EC
:10207000FA0000004C6F6164696E672066726F6DD4
:1020800020454550FA000000427265616BFA00007D
:10209000467265653A2070616765733A0000206397
:1020A000686172733A000000FA496E766F6B696E70
:1020B0006720626F6F746C6F616465722061742059
:1020C000307800004572726F72200000FB303A20B9
:1020D000556E6B6E6F776E20636F6D6D616E6420F1
:1020E0006F72206F70657261746F722E0000FB3129
:1020F0003A20456E636F756E746572656420612069
:1021000076616C75652074686174206973206E6FE8
:1021100074206265747765656E203020616E64207E
:102120003235352E0000FB323A2050726F677261F3
:102130006D206D656D6F72792069732066756C6CAA
:102140002E000000FB333A20456E636F756E746598
:1021500072656420612063686172616374657220D6
:1021600074686174206973206E6F742061207265D9
:10217000636F676E697A656420747970652E0000FC
:10218000FB343A696E7465726E616C206572726FB1
:1021900072202D20627566666572206C696D6974A7
:1021A000206578636565646564000000FB353A204E
:1021B000496E617070726F707269617465207661CA
:1021C000726961626C65206E616D6520656E636F1A
:1021D000756E74657265642E0000FB363A204461AA
:1021E000746120737461636B20707573682065720D
:1021F000726F72202D20746F6F206D616E79206177
:102200007267756D656E7473206F6E206F6E6520DA
:102210006C696E652E000000FB373A2044617461E2
:1022200020737461636B20706F70206572726F72BF
:102230002EFAF9092046756E6374696F6E20747208
:1022400069656420746F2075736520612076616C08
:102250007565207468617420776173206E6F7420D7
:10226000617661696C61626C652E0000FB383A2012
:102270004D616368696E6520737461636B2065727C
:10228000726F72FAF9092046756E6374696F6E7326
:1022900020616E642F6F722063616C6C73206E65B9
:1022A0007374656420746F6F20646565706C792049
:1022B0006F7220746F6F20636F6D706C65780000B3
:1022C000FB393A20474F544F206F7220474F5355E8
:1022D000422064657374696E6174696F6E206C6905
:1022E0006E6520776173206E6F7420666F756E6403
:1022F0002E000000FB413A205370656369666965F2
:10230000642062697420706F736974696F6E2072E3
:10231000616E6765206F6620303A372065786365A7
:10232000656465640000FB423A204C696E65206E6E
:10233000756D62657220686173206D6F72652074BF
:1023400068616E207468726565206E756D65726176
:102350006C730000FB433A205370656369666965DE
:10236000642062697420706F736974696F6E207283
:10237000616E6765206F6620303A3120657863654D
:10238000656465640000FB443A20537065636966C8
:102390006965642062697420706F736974696F6E17
:1023A0002072616E6765206F6620303A3320657851
:1023B0006365656465640000FB453A20496E70758D
:1023C00074204361707475726520726567697374F7
:1023D0006572206F766572666C6F77000000FB4651
:1023E0003A2041726974686D65746963206F76651F
:1023F00072666C6F77000000FB31303A20417269E1
:1024000074686D6574696320756E646572666C6F5F
:1024100077000000FB31313A204469766964652019
:102420006279207A65726F000000FB31323A2054E5
:10243000574920627573206572726F72206F6363F3
:10244000757265640000FB31333A205457492069A6
:102450006E74657266616365206E6F7420656E616F
:10246000626C65640000FB31343A205457492053B4
:102470006C617665207265706C696564207769743B
:1024800068204E414B000000FB31353A204E6F2052
:10249000426F6F742D6C6F6164657220666F756E2C
:1024A00064000000000000000000000000000000C8
:1024B000000000000000000000000000000000001C
:1024C000000000000000000000000000000000000C
:1024D00000000000000000000000000000000000FC
:1024E00000000000000000000000000000000000EC
:1024F00000000000000000000000000000000000DC
:1025000000000000000000000000000000000000CB
:1025100000000000000000000000000000000000BB
:1025200000000000FFFFFFFFFFFFFFFFFFFFFFFFB7
:10253000FFFFFFFFFFFFFFFFFFFFFFFFFFFFFFFFAB
:10254000FFFFFFFFFFFFFFFFFFFFFFFFFFFFFFFF9B
:10255000FFFFFFFFFFFFFFFFFFFFFFFFFFFFFFFF8B
:10256000FFFFFFFFFFFFFFFFFFFFFFFFFFFFFFFF7B
:10257000FFFFFFFFFFFFFFFFFFFFFFFFFFFFFFFF6B
:10258000FFFFFFFFFFFFFFFFFFFFFFFFFFFFFFFF5B
:10259000FFFFFFFFFFFFFFFFFFFFFFFFFFFFFFFF4B
:0425A000FFFFFFFF3B
:00000001FF
